:020000020000FC
:100000000AC05DC05CC0189540C018951895189539
:100010001895189518950FED0DBF01E907BB00E382
:1000200001BB0CE002BB17D0C09A0AE005BF00EC90
:100030000BBF00E101BD09E301BD00E00FBD0DE014
:100040000EBD01E00BBD08E30ABD00E409BF40E0BE
:1000500078940000FECF8D98959A8C9A9498000021
:1000600000008D98859B0FC0A89500E101BD0DE1B2
:1000700001BDF89400E007BB08BB01BB02BB00E771
:1000800005BF889508958D9A08950F930FB70F9324
:100090001F93C798403011F04A95C79AC4980196AB
:1000A00090FF08C0C49A02B30F7C102F106112BBDE
:1000B000000002BB1F910F910FBF0F9118950F9376
:1000C0000FB70F9340E5A8950F910FBF0F911895AB
:00000001FF
